:100D18007584008551D28552D37584018553D28557
:100D280054D3E4F552F5513008068555518556528D
:100D380030090CE5512557F551E5523558F5523033
:100D48000A10E5338534F0A42551F551E5F0355204
:100D5800F552300B10E50A8537F0A42551F551E519
:100D6800F03552F552300C10E5118536F0A42551B6
:100D7800F551E5F03552F552E4F554F553301010BD
:100D8800855553855654E556C3953B4003853B54DA
:100D9800301116E558C3953A4003853B58E553256D
:100DA80057F553E5543558F554301210E53385346A
:100DB800F0A42553F553E5F03554F554301310E5F8
:100DC8000A8537F0A42553F553E5F03554F554302A
:100DD8001410E5118536F0A42553F553E5F0355484
:100DE800F554301510E5188535F0A42553F553E56D
:100DF800F03554F554301610E5288539F0A42553FC
:100E0800F553E5F03554F554301710E5298538F0D9
:100E1800A42553F553E5F03554F554E554C3953CF2
:100E28004003853C5422900E95303103120E503009
:070E38003203120E6030349A
:100E3F0003120E84303303120E83303503120E94D7
:100E4F0022E50B2509F50BE50C3508F50C93F50A92
:100E5F0022E512250EF512E513350DF51393C31385
:100E6F00F8E5142510F514E515350FF51593C31393
:100E7F0028F5112222E5192517F519E51A3516F56A
:100E8F001A93F51822227F8285888C8F9295989BD2
:100E9F009EA1A4A7AAADB0B3B6B9BBBEC1C3C6C904
:100EAF00CBCED0D3D5D7D9DCDEE0E2E4E6E7E9EB71
:100EBF00EDEEF0F1F2F4F5F6F7F8F9FAFBFCFCFDC4
:100ECF00FDFEFEFEFEFEFEFEFEFEFEFDFDFCFCFB3D
:100EDF00FAFAF9F8F7F6F4F3F2F0EFEDECEAE8E7E7
:100EEF00E5E3E1DFDDDBD8D6D4D1CFCDCAC8C5C2AB
:100EFF00C0BDBAB7B4B2AFACA9A6A3A09D9A979440
:100F0F00908D8A8784817E7A7774716E6B68656243
:100F1F005F5C595653504D4A4744423F3C39373432
:100F2F00322F2D2A282624211F1D1B1918161412A3
:100F3F00110F0E0C0B0A0807060504040302020129
:100F4F000100000000000000000000010102020388
:100F5F000405060708090A0B0D0E101113151618B4
:100F6F001A1C1E20222427292B2E303335383A3DC8
:100F7F00404245484B4E515456595C606366696C0C
:060F8F006F7275787B7F94
:10146F00D2F4C2F5C2F675840F85F0C812129F74BC
:10147F00031214BE12129374031214BE12127612B8
:10148F00127674031214BE12127674021214BE1264
:10149F001276742812152A740612152A740E121554
:1014AF002A740112152A121293748012152A22C05F
:1014BF0000A2E092F3A2E192F2A2E292F1A2E392F1
:1014CF00F0D2F475840F85F0C8C2F47830D8FE8559
:1014DF00F0C87830D8FED00022C00075840FA2E487
:1014EF0092F3A2E592F2A2E692F1A2E792F0D2F481
:1014FF0085F0C8C2F47830D8FE85F0C87830D8FEB1
:10150F00D00022EF75840FD2F5C2F685F0C8121401
:10151F00E81212761214BE1212762275840FC2F5DB
:10152F00C2F685F0C81214E81212761214BE121207
:10153F007622EF14A2E492E6C2E4D2E712152A2231
:10154F00740F12152A22740D12152A227F011215FB
:10155F004178107F20121512D8F9227F11121541F0
:10156F0078107F20121512D8F9227F0112154178B9
:10157F00207F20121512D8F922C0077F018004C0E6
:10158F00077F11121541D007C082C083C007EF75C6
:10159F00F0109015B91212B77810E493FF121512CC
:0915AF00A3D8F7D007D083D08245
:1015B8002220202020202020202020202020202021
:1015C8002030313233343536373839414243444597
:1015D8004620202052533432322054455354202080
:1015E8002020202052533233322054455354202097
:1015F8002020205445535420204641494C4544203E
:101608002020205445535420205041535345442012
:10161800202020454550524F4D20544553542020FA
:1016280020204155582052454C4159205445535487
:101638002020205055534820544F2054414C4B20D3
:101648002054455354203320434841522F53554288
:101658002054455354204649584544205354524930
:101668004E544553542056415249422053545249EE
:101678004E464143544F52592044454641554C54D7
:101688002050524F4752414D4D494E47204D4F44EF
:101698004553494D504C45582052455045415445B5
:1016A800522020205245434F5244494E4720202083
:0116B8002011
:10374E00C2B6758400D2C2C2C6D2C6C2C4D2C5C267
:10375E00C330C3FD74A0F5C2C2C5C2C330C3FD8E53
:10376E00C2C2C330C3FD8FC2C2C330C3FD8DC2C23D
:10377E00C330C3FDD2C4C2C320C4FD121293D2B64D
:10378E0022758400C2C3D2C530C3FD74A0F5C2C277
:10379E00C5C2C330C3FD8EC2C2C330C3FD8FC2C209
:1037AE00C330C3FDC2C4D2C5C2C330C3FD74A1F5BC
:1037BE00C2C2C5C2C330C3FDC2C2C2C330C3FD85BF
:0A37CE00C207D2C4C2C320C4FD220A
:080003000216B9000000000024
:08000B000216BA00000000001B
:08001300021835000000000096
:08001B003200000000000000AB
:09002300320000000000000000A2
:08002B000216BD0000000000F8
:08003300320000000000000093
:0A003B003200000000000000000089
:0900430032000000000000000082
:08004B0032000000000000007B
:08005300320000000000000073
:08005B0002171C000000000068
:08006300320000000000000063
:08006B0002173A00000000003A
:080073000216C30000000000AA
:08007B0002183600000000002D
:08008300021719000000000043
:08008B0032000000000000003B
:1000930002185400000000000000000000000000EF
:1000A3003275FF0775FFDE75FFAD75840F75E107C8
:1000B30075E20475E34475840F75A43575A5097558
:1000C300A6FF75A7FF759CFF759D00759E00759F24
:1000D300F075D8FF75E8FF75F80F75AD0F758401DE
:1000E30075893075888F75840275893075888F7529
:1000F300840F758A80758C67780874FF0000000090
:100103000000000000000000D5E0F1D8EDE58C30E0
:10011300E7FB759701758A0043890475840075B7F9
:100123001075840F438901758D01758F01758E02DA
:100133007480D5E0FD438902E58930E4FB759702BD
:1001430075840075D10775840075BB0175BA007598
:10015300BCF075C70075C60075C5FF75C4FF75E8AB
:100163008175840275BB0475BA0075BCF175C60050
:1001730075C4FF75E88875840075D484758401752A
:10018300D484758400C2F8759A47759D1A43F8099B
:1001930075870075840075B90075A90075910075A0
:1001A300985075840175981075840075C04075C3A7
:1001B3000075CFC9758400758E0075892075880513
:1001C300758400758A00758B6F758CF4758D6F431C
:1001D300885075840075C90075CA0075CB0075CC4D
:1001E3000075CD0075C80075840175C91875CA807E
:1001F30075CBFB75CDFB75CC80D2CA75840275C9EE
:100203001875CA1275CBF775CDF775CC12D2CA75AE
:10021300840075A8AF75B80075E6A475E71775F681
:100223000075F7019000007F007E20E4F0A3DFFC5F
:02023300DEFAF1
:100235007534FF7535FF7536FF7537FF7538FF75F2
:0C02450039FF753AFF753BFF753CFF2246
:1016B90032C28D32758400C2CF32C0E0C083C0828D
:1016C900C0D0C000C0F0C2CFB237203723120D18E6
:1016D900151BE51B7009751B0A7584017588AF1503
:1016E9001CE51C7009751C607584027588AF800E35
:1016F900120E2E152AE52A7005752A04D28B7584D7
:1017090000D2ECD0F0D000D0D0D082D083D0E0325B
:10171900C2CF32C0E0C0D0E52B6002152BE52E60A8
:1017290002152EE55E6002155E75888FD0D0D0E077
:1017390032C0E0C0D0C084202E1375840F30DF255D
:10174900E5E8540FF53DD22E753EC88018153EE5E3
:101759003E7006E53DD2E7F53D75840F20DF06C2F0
:101769002ED22DD22920301475840F30F826E5E8C1
:1017790054F0C4F53FD2307540C880181540E54093
:101789007006E53FD2E7F53F75840F20F806C230B1
:10179900D22FD228E52C6002152CE55B6002155B7F
:1017A900E55D6002155DE56560021565B2A1151D6F
:1017B900E51D706F751D0AE52D6002152DE55F6049
:1017C90002155FE52F6002152FE56060021560E5DF
:1017D9006160021561E55960021559E55A60021503
:0D17E9005AE54E6002154EE54F6002154FA7
:1017F600E55060021550E56360021563151EE51E8F
:101806007024751E0AE55C6002155CE564600215CD
:1018160064E56660021566151FE51F7009751F06EB
:10182600E56260021562D084C28DD0D0D0E032323B
:10183600202C0DD22C85BF5885BE5775BB01800B59
:10184600C22C85BF5685BE5575BB00C2ED32C0E0C1
:10185600C0D0E541B4000D054185BE3375BCF175B8
:10186600BB07804CB4010D054185BE308542BC7571
:10187600BB04803CB4020D054185BE3375BCF175D1
:10188600BB06802CB4030D054185BE318542BC756F
:10189600BB04801CB4040D054185BE3375BCF175CF
:1018A600BB05800C75410085BE328542BC75BB0404
:0718B600C2EDD0D0D0E032FA
:1012060075840FD2FD2275840FC2FD2275840FD21C
:10121600FC2275840FC2FC2275840FD2FED21C22DA
:1012260075840FC21CC2FE22C29322D293227584F9
:101236000FA2FA2275840FA2F92275840FA2DD226D
:1012460075840FA2DE22A2922275840FA2DA22757D
:10125600840FA2DB2275840FA2D82275840FA2D92F
:101266002200000000000000000000000000002234
:10127600C000C001790478B4D8FED9FAD001D000F4
:1012860022C0007814121276D8FBD00022C0E07576
:101296002B05E52B70FCD0E022C0E0752B0FE52B6B
:1012A60070FCD0E022C0E0752B64E52B70FCD0E02A
:1012B60022A42582F582E58335F0F58322B40A005F
:1012C60022C0E0C3997001D3D0E022B506012250B6
:1012D60007B5070122400122D322EF75F06484246A
:1012E60030900061F0E5F0A375F00A842430F0A395
:1012F600E5F02430F022EF75F0648424309000612C
:07130600F0E5F0A375F00A09
:10130D00842430F0A3E5F02430F0900061E0B43097
:10131D000B7420F0A3E0B430037420F02290000E83
:10132D00E0540FFFA3E0B420028019540FCF75F0E5
:10133D000AA42FFFA3E0B420028009540FCF75F04B
:10134D000AA42FFF22C006C005C00490000EE05471
:10135D000FFFFEA3E0B42003C3802C540FFDCF7507
:10136D00F00AA42FFFA3E0B42003C3801A540FFC8E
:10137D00EE75F064A420D20EFEED75F00AA42E4099
:10138D00052C40028001D3D004D005D0062275F083
:10139D006484F6E5F00875F00A84F608A6F00822D4
:1013AD00C0017900E6B4FF028027F908E6B4FF0317
:1013BD00C38022E975F00AA426F908E6B4FF03C339
:1013CD008013E975F00AA420D207C3264003F980E3
:1013DD0004D3D00122E9D00122E675F00AA4082633
:1013ED00227846EE12139B7544007545007848909F
:0413FD001447790810
:10140100EF134007A3A3A3A3A3801CC0E0C000C0A7
:1014110001C37905E49336D4A2E4540FF6A318D995
:10142100F3D001D000D0E0D9D8E544600C7545096E
:1014310075460975470975480985454485464585B9
:1014410047468548472206050200000201050000C3
:101451000402000100080400020006090004000261
:0E14610009010800040803060108060702033B
:1002510044313233343536373839302A2341424339
:1002610044AAA3C1C2C3C4D7ABA8A92A234142430C
:100271000101010101010101010000000000000074
:10028100000000000000000000000000000000006D
:10029100000000000000000000000000000000005D
:1002A100000000000000000000000000000000004D
:1002B100000000000000000000000000000000003D
:1002C1000000000000000000000001010101010127
:1002D100010101000000000000000000000000001A
:1002E100000000000000000000000000000000000D
:1002F10000000000000000000000000000000000FD
:1003010000000000000000000000000000000000EC
:1003110000000000000000000000000000000000DC
:1003210000000000010101010101010101000000C3
:1003310000000000000000000000000000000000BC
:1003410000000000000000000000000000000000AC
:10035100000000000000000000000000000000009C
:10036100000000000000000000000000000000008C
:10037100000000000000000000000000000001017A
:100381000101010101010100000000000000000065
:10039100000000000000000000000000000000005C
:1003A100000000000000000000000000000000004C
:1003B100000000000000000000000000000000003C
:1003C100000000000000000000000000000000002C
:1003D1000000000000000000010101010101010114
:1003E100010000000000000000000000000000000B
:1003F10000000000000000000000000000000000FC
:1004010000000000000000000000000000000000EB
:1004110000000000000000000000000000000000DB
:1004210000000000000000000000000000000000CB
:1004310000000101010101010101010000000000B2
:1004410000000000000000000000000000000000AB
:10045100000000000000000000000000000000009B
:10046100000000000000000000000000000000008B
:10047100000000000000000000000000000000007B
:1004810000000000000000000000000020202020EB
:10049100202020202020202020202020202020205B
:1004A100202020202020202020202020202020204B
:1004B100202020202020202020202020202020203B
:1004C100202020202020202020202020202020202B
:1004D100202020202020202020202020202020201B
:1004E100202020202020202020202020202020200B
:1004F10020202020202020202020202020202020FB
:1005010020202020202020202020202020202020EA
:1005110020202020202020202020202020202020DA
:1005210020202020202020202020202020202020CA
:1005310020202020202020202020202020202020BA
:1005410020202020202020202020202020202020AA
:10055100474C4F42414C202020202020204354432F
:10056100535320434F444520202020202020444342
:100571005320434F44452020202020204C5452201A
:100581005245504541544552202020205350454565
:1005910044204449414C494E472020205350454571
:1005A100442043414C4C494E472020202050544385
:1005B100204E554D424552202020202020564F49A3
:1005C1004345204D455353414745532020564F49FC
:1005D100434520504C41594241434B202020494E34
:1005E10056414C49442054595045202020204F5514
:1005F10054204F462052414E4745202020494C4C23
:100601004547414C2056414C554520204D555354AA
:100611002046494C4C204649454C44202020494C19
:100621004C4547414C20434F4445202020444154F0
:100631004120414343455054454420204C494E45B7
:10064100204E554D4245523A2020202055534552C7
:100651002050524F4752414D4D494E4755534552F7
:100661002049443A2020202020202020564F494371
:1006710045205245434F5244494E472020494C4C56
:100681004547414C20454E545259202020494C4C5D
:100691004547414C2047414E472020202020204300
:1006A1004F4D504C455445442020202036333036A0
:1006B10037303639343731393734343737303739E1
:1006C10037383235383534383835393135393438C9
:1006D10039373431303031303331303731313031F5
:1006E10031343131383132333132373133313133E1
:1006F10036313431313436313531313536313539C0
:1007010031363231363531363731373131373331B0
:100711003737313739313833313836313839313982
:100721003231393631393932303332303632313093
:100731003231383232353232393233333234313286
:100741003530323534303036303037303135303184
:100751003730323130323330323530323630333176
:100761003033323033363034333034373035303063
:100771003531303533303534303635303731303747
:10078100323037333037343131343131353131363C
:100791003132323132353133313133323133343137
:1007A1003431313433313435313532313535313518
:1007B1003631363231363531373231373432303500
:1007C1003231323231343232333232353232363200
:1007D10034333234343234353234363235313235E1
:1007E10032323535323631323633323635323636CB
:1007F10032373132373433303633313133313533C7
:1008010032353333313333323334333334363335B2
:10081100313335363336343336353337313431319C
:10082100343132343133343233343331343332349A
:100831003435343436343532343534343535343670
:100841003234363434363534363635303335303665
:100851003531363532333532363533323534363556
:100861003635363036363132363234363237363343
:100871003136333236353436363236363437303334
:100881003731323732333733313733323733343725
:1008910034333735344142434445464748494A4B4E
:1008A1004C4D4E4F505152535455565758595A6109
:1008B10062636465666768696A6B6C6D6E6F70719F
:1008C10072737475767778797A303132333435369C
:1008D100373839607E21402324255E262A28295F66
:1008E1002D2B3D7B7D5B5D7C3A3B3C3E2C2E3F2F8F
:1008F1002020202020202020206401001102211529
:1009010001016402001103211501016404001104B5
:100911002115010164080011052115010178060165
:1009210011060119010182030711072515057882B6
:100931000208110824150A6382020911092315000E
:100941006382020A110A2315006382020B110B2430
:1009510015006382030C110C261500FF82030D1193
:100961000D261500FF82010E110E271500028201CE
:100971000F110F27150002820310111026150AFF0F
:100981008203111111261500FF820312111226157F
:1009910000FF8203131113261500FF8202141114A4
:1009A10022150063820215111524150063641000DD
:1009B100111621150101642000111728150101826A
:1009C10003161118261500FF6440001119011501C5
:1009D10001820217111A24150063820218111B24C7
:1009E100150063820119111C291500026480001190
:1009F1001D2815010182031A111E261500FF780416
:100A01001B111F2A17010178041F11202A17010148
:100A1100820123112B21150001820324112C25159C
:100A210000FF202020202020202020202020202006
:100A310020202020202020202020202020202020B5
:100A410020202054454C434F2050524F4752414D96
:100A5100202020524144494F2050524F4752414D8E
:100A610020202050484F4E452050524F4752414D73
:100A7100202020434F4D50552050524F4752414D59
:100A81002020202041434345535320434F444520D8
:100A910020204D4158205245504541542054494D44
:100AA10045202056414C4944204D4553534147452B
:100AB1002020205455524E204F4E2044454C415940
:100AC1002020205455524E204F46462044454C414B
:100AD10059205455524E2041524F554E4420444CBA
:100AE100592044544D462054454C434F204C4556C3
:100AF100454C44544D4620524144494F204C4556A3
:100B0100454C2020564F49434520505245414D50B8
:100B1100202020525820505245414D5020474149F4
:100B21004E20564F49434520584D4954204C455677
:100B3100454C2054574F20544F4E45204C45564567
:100B41004C204245455020524144494F204C455686
:100B5100454C424545502054454C434F204C455649
:100B6100454C434F53204143515549542054494D1D
:100B71004520434F532052454C454153452054494C
:100B81004D45494E5445524E414C20535155454CCB
:100B910043482020434F5320504F4C415249545910
:100BA1002020434F53205452494747455220564F26
:100BB1004C5454574F20544F4E4520454E41424CC2
:100BC100452020205245434F52442044454C415931
:100BD1002020202052454144592044454C41592070
:100BE10020204E554D424552204F4620544F4E45F0
:100BF10053202053454E534520504F4C41524954A8
:100C0100592053454E5345205452494720564F4C85
:100C110054202054574F20544F4E452053454E5396
:100C21004520202054574F20544F4E4520434F53C9
:100C31002020202020202020202020202020313D85
:100C4100454E20202020202020202020202031203F
:100C51004D53202020202020202020202031302012
:100C61004D532020202020202020202031303020F2
:100C71004D532020202020202020202020202053E0
:100C81004543202020202020202020202052415494
:100C9100494F202020202020202020202054414284
:100CA1004C452020202020202020202020313D5094
:100CB1004F532020202020202020202020204E4D76
:100CC1004252202020202020202020202020544F6C
:100CD1004E45202042555359204348414E4E454CE4
:100CE100202020504C41594241434B2044454C4126
:100CF1005920AF313233343536780A0A6314FF3262
:100D01000101FFFF3232000A8000140180303130CE
:070D110032303230330000E4
:104C6C00756264E4900000F0301E0B301D24124875
:104C7C00591218BD80F5301F0B301D1612489812B2
:104C8C0018BD80F530200B301D08121E561218BDB1
:034C9C0080F5227E
:1018BD00E5627012900000E0D394004009C21EC290
:1018CD001FC220C21D22900000E012324919D4001F
:1018DD0019D70119DA0219DD0319E00419E2051906
:1018ED00E40619E60719E90819EC0A19EF0B19F2C4
:1018FD000F19F51019F81419FB1519FE191A011AFB
:10190D001A041B1A071E1A0A1F1A0D231A10241A5D
:10191D0013281A16291A192D1A1C2E1A1F2F1A22BE
:10192D00301A25321A28331A2A341A2D351A3064F2
:10193D001A33651A36661A39671A3C6E1A3E6F1AD3
:10194D0040701A82711A42781A44791A467A1A82AC
:10195D007B1A48821A4A831A4C841A4E851A518C66
:10196D001A548D1A568E1A588F1A5B961A5E971A3C
:10197D0060981A62991A65A01A68A11A6BA21A6D5D
:10198D00A31A70AA1A72AB1A75AC1A77AD1A7AB47B
:10199D001A7DB51A80B61A82B71A84BE1A87BF1A75
:1019AD008AC01A8DC11A82C21A93F01A96F11A9929
:1019BD00F21A9CFA1A9FFB1AA2FC1AA5FD1AA8FE90
:1019CD001AABFF00001AAE0254A502525E02471078
:1019DD00025042800480028000024634021FC4027D
:1019ED004CD20223EC02431C02253A02437102261B
:1019FD00880247DB0240A2022BC00244B60227D662
:101A0D00024503022924024550022A72024DF702B3
:101A1D004B2802467E1245E90241BA8000023D0F75
:101A2D000247980243C6024754024B61024214809A
:101A3D00468032804B804080228045800780268002
:101A4D003F02459D023331801C8035024417023818
:101A5D00E18008802B02481A0234B1023CA080209C
:101A6D000233F18012023A54801602229302395E3B
:101A7D00023D7D800B800C023B460244670236B16D
:101A8D000249530242C6025069023DE60254D20297
:101A9D00426E025593025594025595023ACD025568
:071AAD0096E4900000F02216
:0F54A500E4900002F0756264900000E004F022D1
:10525E0012155B12156A7BFF7A06794D124D097F86
:0F526E0011121541C224C221900000E004F02269
:10471000302140900001E0FFC221BF2A0790000035
:10472000E004F022EF6423702A7F23121512900018
:1047300002E004F0E0C394034013C21EC21FC22073
:10474000C21DE4900000F01250180239DA90000007
:034750007402F000
:014753002243
:105042007BFF7A06794D124D0912156A7F111215EE
:105052004112550AE490003DF07F2A121512C22433
:07506200900000E004F022C1
:10463400302146900001E0F569C221E569642A60F1
:1046440038AF691254B45022AF6912151290003D6C
:10465400E02404F582E43400F583E569F090003D3C
:10466400E004F0900000E004F0227BFF7A06797DFC
:09467400124D0990000074FAF0E7
:01467D00221A
:101FC40020210302212E900001E0FFC221BF2A0735
:101FD4009000007403F022EF6423600302211F12B7
:101FE4001512900005E064397077A3E064397071CC
:101FF400A3E06439706BD226900004E0FFB431088A
:10200400E4900037F002208EEFB43208E4900038F8
:10201400F00220A1EFB43302803E900004E0FFB44C
:102024003408E4900039F00220CFEFB43508E4908E
:10203400003AF00220E5EFB43608E490003BF002E9
:1020440020FBEFB437028010900004E0B438028023
:1020540007900004E0B4390B7BFF7A06798D0221E6
:1020640025C226900004E0FFB43016A3E0B430117A
:10207400A3E0B4300CA3E0B43007900000740AF07D
:1020840022EFB4310C1241015007900000740FF09C
:1020940022900004E0B4320C124042500790000039
:1020A4007414F022900004E0B43311A3E0B4300CB3
:1020B4001251DC50079000007419F022900004E0E3
:1020C400B4340FA3E0B4300A125376900000741EA7
:1020D400F022900004E0B4350FA3E0B4300A1253A8
:1020E4008B9000007423F022900004E0B4360FA318
:1020F400E0B4300A1253A09000007428F02290003B
:1021040004E0B43716A3E0B43011A3E0B4300CA358
:10211400E0B43007900000742DF0227BFF7A06793A
:0A2124007D124D0990000074FAF0DE
:01212E00228E
:104CD20090003C740BF090003D7407F0E490004E9D
:104CE200F090004FF0900050F07BFF7A05794D1262
:104CF2004D09124D347F1E1215419000007432F09E
:014D0200228E
:1023EC00123BBBD3900067E09421900066E0940010
:1023FC00400A124D0390000074FAF022900066E03F
:10240C00FEA3E0FF9008FA75F00912323DEE75F06C
:10241C0009A42583F583E493900045F09008FB759F
:10242C00F009EF12323DEE75F009A42583F583E433
:10243C0093900046F0900066A3E09008FC75F009BC
:10244C0012323DEE75F009A42583F583E4939000D8
:10245C0047F09008FD75F009EF12323DEE75F0096A
:10246C00A42583F583E493900048F0900066A3E0E4
:10247C009008FE75F00912323DEE75F009A4258323
:10248C00F583E493FD900049F09008FF75F009EF97
:10249C0012323DEE75F009A42583F583E493900088
:1024AC004AF0900066A3E090090075F00912323DE5
:1024BC00EE75F009A42583F583E49390004BF0901E
:1024CC00090175F009EF12323DEE75F009A4258370
:1024DC00F583E49390004CF0900066A3E090090221
:1024EC0075F00912323DEE75F009A42583F583E4ED
:1024FC009390004DF0ED6015900049E075F010A43C
:10250C002423F9740A35F0FA7BFF124D0990004A26
:10251C00E0FF601175F010A42423F9740A35F0FA69
:0E252C007BFF124D3A900045E0900000F02237
:10431C0090003C7410F090003D7407F090004E74C7
:10432C00C8F090004F740AF0900037E0900050F005
:10433C007BFF7A05795D124D09124D347F0D1215F4
:10434C0041900005E0FF121512900006E0FF1215D7
:10435C0012900007E0FF1215127F1E1215419000FB
:05436C00007432F02294
:10253A00123BBBD3900067E09400900066E09400E1
:10254A00400A124D0390000074FAF022900066E0EF
:10255A00FEA3E0FF90027175F00912323DEE75F0AC
:10256A0009A42583F583E493900045F090027275DF
:10257A00F009EF12323DEE75F009A42583F583E4E4
:10258A0093900046F0900066A3E090027375F009FC
:10259A0012323DEE75F009A42583F583E493900089
:1025AA0047F090027475F009EF12323DEE75F009AA
:1025BA00A42583F583E493900048F0900066A3E095
:1025CA0090027575F00912323DEE75F009A4258363
:1025DA00F583E493FD900049F090027675F009EFD7
:1025EA0012323DEE75F009A42583F583E493900039
:1025FA004AF0900066A3E090027775F00912323D26
:10260A00EE75F009A42583F583E49390004BF090CE
:10261A00027875F009EF12323DEE75F009A42583B0
:10262A00F583E49390004CF0900066A3E090027961
:10263A0075F00912323DEE75F009A42583F583E49D
:10264A009390004DF0ED6015900049E075F010A4EC
:10265A00248DF9740435F0FA7BFF124D0990004A73
:10266A00E0FF601175F010A4248DF9740435F0FAB6
:0E267A007BFF124D3A900045E0900000F022E8
:1043710090003C7415F090003D7407F090004E746D
:104381002CF090004F740AF0900038E0900050F04B
:104391007BFF7A05796D124D09124D347F0C121590
:1043A10041900005E0FF121512900006E0FF121582
:1043B10012900007E0FF1215127F1E1215419000A6
:0543C100007432F0223F
:10268800123BBBD3900067E09400900066E0940092
:10269800400A124D0390000074FAF022900066E0A0
:1026A800FEA3E0FF9002CB75F00912323DEE75F003
:1026B80009A42583F583E493900045F09002CC7536
:1026C800F009EF12323DEE75F009A42583F583E495
:1026D80093900046F0900066A3E09002CD75F00953
:1026E80012323DEE75F009A42583F583E49390003A
:1026F80047F09002CE75F009EF12323DEE75F00901
:10270800A42583F583E493900048F0900066A3E045
:102718009002CF75F00912323DEE75F009A42583B9
:10272800F583E493FD900049F09002D075F009EF2D
:1027380012323DEE75F009A42583F583E4939000E9
:102748004AF0900066A3E09002D175F00912323D7C
:10275800EE75F009A42583F583E49390004BF0907F
:1027680002D275F009EF12323DEE75F009A4258307
:10277800F583E49390004CF0900066A3E09002D3B8
:1027880075F00912323DEE75F009A42583F583E44E
:102798009390004DF0ED6015900049E075F010A49D
:1027A80024ADF9740435F0FA7BFF124D0990004A04
:1027B800E0FF601175F010A424ADF9740435F0FA47
:0E27C8007BFF124D3A900045E0900000F02299
:1047DB007BFF7A05797D124D097BFF7A06795D1295
:1047EB004D3A7F0E121541900006E0FF1215129004
:1047FB000007E0FF1215127F1A12154190003C744E
:0F480B001AF090003D7404F09000007432F02217
:1040A2003027079000007403F022124D347F1E1255
:1040B2001541123E4E900068E0FEA3E0FFD394004B
:1040C200EE94004030EF94FBEE9400502890003CB8
:1040D200741BF090003D7407F090004E745EF090F7
:1040E200004F740AF0900036E014900050F09000F7
:0F40F200007432F022124D0390000074FAF02295
:102BC000D3900067E09400900066E09400400A1201
:102BD0004D0390000074FAF022900066E0FEA3E03E
:102BE000FF90032575F00912323DEE75F009A4251A
:102BF00083F583E493900045F090032675F009EF88
:102C000012323DEE75F009A42583F583E49390001C
:102C100046F0900066A3E090032775F00912323D5C
:102C2000EE75F009A42583F583E493900047F090B6
:102C3000032875F009EF12323DEE75F009A42583E3
:102C4000F583E493900048F0900066A3E090032998
:102C500075F00912323DEE75F009A42583F583E481
:102C600093FD900049F090032A75F009EF12323D70
:102C7000EE75F009A42583F583E49390004AF09063
:102C80000066A3E090032B75F00912323DEE75F05B
:102C900009A42583F583E49390004BF090032C75F1
:102CA000F009EF12323DEE75F009A42583F583E4B7
:102CB0009390004CF0900066A3E090032D75F0090E
:102CC00012323DEE75F009A42583F583E49390005C
:102CD0004DF0ED6015900049E075F010A424CDF999
:102CE000740435F0FA7BFF124D0990004AE0FF6052
:102CF0001175F010A424CDF9740435F0FA7BFF129D
:0B2D00004D3A900045E0900000F022EA
:1044B60090003C741FF090003D7407F090004E741D
:1044C60090F090004F740AF0900039E0900050F0A0
:1044D6007BFF7A05798D124D09124D347F0F121527
:1044E60041900006E0FF121512900007E0FF12153A
:0D44F600127F1E1215419000007432F0225A
:1027D600123BBBD3900067E09400900066E0940043
:1027E600400A124D0390000074FAF022900066E051
:1027F600FEA3E0FF90037F75F00912323DEE75F0FF
:1028060009A42583F583E493900045F09003807531
:10281600F009EF12323DEE75F009A42583F583E445
:1028260093900046F0900066A3E090038175F0094E
:1028360012323DEE75F009A42583F583E4939000EA
:1028460047F090038275F009EF12323DEE75F009FC
:10285600A42583F583E493900048F0900066A3E0F6
:1028660090038375F00912323DEE75F009A42583B5
:10287600F583E493FD900049F090038475F009EF29
:1028860012323DEE75F009A42583F583E49390009A
:102896004AF0900066A3E090038575F00912323D78
:1028A600EE75F009A42583F583E49390004BF09030
:1028B600038675F009EF12323DEE75F009A4258303
:1028C600F583E49390004CF0900066A3E0900387B4
:1028D60075F00912323DEE75F009A42583F583E4FF
:1028E6009390004DF0ED6015900049E075F010A44E
:1028F60024EDF9740435F0FA7BFF124D0990004A75
:10290600E0FF601175F010A424EDF9740435F0FAB7
:0E2916007BFF124D3A900045E0900000F02249
:1045030090003C7424F090003D7407F090004E74CA
:10451300F4F090004F740AF090003AE0900050F0ED
:104523007BFF7A05799D124D09124D347F0F1215C9
:1045330041900006E0FF121512900007E0FF1215EC
:0D454300127F1E1215419000007432F0220C
:10292400123BBBD3900067E09400900066E09400F3
:10293400400A124D0390000074FAF022900066E001
:10294400FEA3E0FF9003D975F00912323DEE75F055
:1029540009A42583F583E493900045F09003DA7588
:10296400F009EF12323DEE75F009A42583F583E4F6
:1029740093900046F0900066A3E09003DB75F009A5
:1029840012323DEE75F009A42583F583E49390009B
:1029940047F09003DC75F009EF12323DEE75F00953
:1029A400A42583F583E493900048F0900066A3E0A7
:1029B4009003DD75F00912323DEE75F009A425830C
:1029C400F583E493FD900049F09003DE75F009EF80
:1029D40012323DEE75F009A42583F583E49390004B
:1029E4004AF0900066A3E09003DF75F00912323DCF
:1029F400EE75F009A42583F583E49390004BF090E1
:102A040003E075F009EF12323DEE75F009A4258359
:102A1400F583E49390004CF0900066A3E09003E10A
:102A240075F00912323DEE75F009A42583F583E4AF
:102A34009390004DF0ED6015900049E075F010A4FE
:102A4400240DF9740535F0FA7BFF124D0990004A04
:102A5400E0FF601175F010A4240DF9740535F0FA47
:0E2A64007BFF124D3A900045E0900000F022FA
:1045500090003C7429F090003D7407F090004E7478
:1045600058F090004F740AF090003BE0900050F03B
:104570007BFF7A0579AD124D09124D347F0D12156E
:1045800041900006E0FF121512900007E0FF12159F
:0D459000127F1E1215419000007432F022BF
:102A7200123BBBD3900067E09400900066E09400A4
:102A8200400A124D0390000074FAF022900066E0B2
:102A9200FEA3E0FF90043375F00912323DEE75F0AB
:102AA20009A42583F583E493900045F090043475DE
:102AB200F009EF12323DEE75F009A42583F583E4A7
:102AC20093900046F0900066A3E090043575F009FB
:102AD20012323DEE75F009A42583F583E49390004C
:102AE20047F090043675F009EF12323DEE75F009A9
:102AF200A42583F583E493900048F0900066A3E058
:102B020090043775F00912323DEE75F009A4258361
:102B1200F583E493FD900049F090043875F009EFD5
:102B220012323DEE75F009A42583F583E4939000FB
:102B32004AF0900066A3E090043975F00912323D24
:102B4200EE75F009A42583F583E49390004BF09091
:102B5200043A75F009EF12323DEE75F009A42583AF
:102B6200F583E49390004CF0900066A3E090043B60
:102B720075F00912323DEE75F009A42583F583E460
:102B82009390004DF0ED6015900049E075F010A4AF
:102B9200242DF9740535F0FA7BFF124D0990004A95
:102BA200E0FF601175F010A4242DF9740535F0FAD8
:0E2BB2007BFF124D3A900045E0900000F022AB
:104DF7003020079000007401F02290003C742EF0E0
:104E070090003D7407F07BFF7A0579BD124D0912BA
:0E4E17004D347F1E1215419000007432F022BF
:104B2800302707900000742FF02290000BE06438C3
:104B38006005A3E0B4390A124D0390000074FAF03E
:104B4800227BFF7A06796D124D0990000BE0540F15
:094B5800F54C9000007430F022CD
:10467E0090000BE064386005A3E0B4390A124D03D4
:10468E0090000074FAF0227BFF7A0579CD124D0965
:10469E0090000BE0540FF54CD20AD21290007CE041
:1046AE00F534121AB47BFF7A06799D124D09C20AAF
:0946BE00C21290000074FEF0220B
:1045E90090000BE0540FF54C301E02D208121AC687
:1045F900301E1B202F04E52F70F9121ABDC2087B4B
:10460900FF7A06799D124D0990000074FEF0301F63
:1046190019202D04E52F70F9121ABD7BFF7A06794E
:0B4629009D124D0990000074FEF0226D
:1041BA00302156900001E0FF900035F0C22112151F
:1041CA0012900035E0FF1254B45021900035E0FF00
:1041DA0090003DE02404F582E43400F583EFF0908A
:1041EA00003DE004F0900000E004F022900035E089
:1041FA00B42A079000007403F0227BFF7A06797DC7
:0A420A00124D0990000074FAF02232
:103D0F0030216A900001E0FF900035F0C2211215BA
:103D1F0012900035E0FFB42A0B90003CE0900000B9
:103D2F00F0D22722EFB4230B90003CE0900000F07C
:103D3F00C22722900035E0FF1254B4502190003575
:103D4F00E0FF90003DE02404F582E43400F583EFBA
:103D5F00F090003DE004F0900000E004F0227BFFC3
:0E3D6F007A06797D124D0990000074FAF02258
:1047980030213F900001E0FF900035F0121512C261
:1047A80021900035E0FFB42A0B90003CE090000017
:1047B800F0D22722EFB4230B90003CE0900000F0E9
:1047C800C227227BFF7A06797D124D09900000747A
:0347D800FAF022D2
:0A43C600900048E0FF700330273834
:1043D00012154112517512378F8F69900046E052C5
:1043E00069E56960047F3180027F30121512302741
:1043F00017C227E5692430900024F090003474013E
:08440000F090000074F0F022BE
:0F44080090004BE0FF121541900000E004F022FD
:10475400302140900001E0FF900035F0C221121595
:1047640012900035E0FFB42A079000007403F02291
:104774001254B4500F900035E090000EF0900000F9
:10478400E004F0227BFF7A06797D124D0990000047
:0447940074FAF022A1
:104B6100302132900001E0FF900035F0C221BF2AD0
:104B7100079000007403F022900035E0B423079001
:104B81000000E004F0227BFF7A06797D124D099046
:064B9100000074FAF0229E
:1042140012517590006AEEF0A3EFF012378F8F6998
:1042240090003E7401F090000EE0B4310890004616
:10423400E04269800E90000EE0B4301E900046E02B
:10424400F4526990006AE0FEA3E0FFAD6912374EB4
:104254001253B590000074FEF0227BFF7A06797D3C
:09426400124D0990000074FAF0FB
:01426D00222E
:103B4600900048E0FF700330275612154112517558
:103B560090006AEEF0A3EFF0E4F569900046E0FF0E
:103B6600E569C39F502790006AE475F00112322779
:103B7600AFF0FE12378F8F6A74242569F582E4341C
:103B860000F583E56AF0121512056980CE3027101C
:103B9600C227E56904900034F090000074F0F0222A
:103BA60090003D740AF090004BE0FF121541900022
:043BB60000E004F037
:013BBA0022E8
:103A5400302175900001E0FF900035F0C22112156D
:103A640012900035E0FFB42A079000007403F0229E
:103A7400EFB42308900000E004F080391254B450ED
:103A840038900035E0FF90003DE0FE04F074042E11
:103A9400F582E43400F583EFF0900046E02409FF5A
:103AA400E433FE90003DE0D39FEE6480F874809888
:103AB4004016900000E004F0227BFF7A06797D1224
:093AC4004D0990000074FAF02293
:10495300302137900001E0FF900035F0C22112159D
:1049630012900035E0FFB42A079000007403F02290
:10497300EFB42307900000E004F0227BFF7A06796E
:0B4983007D124D0990000074FAF02234
:1042C60012517590006AEEF0A3EFF090003D740A6B
:1042D600F0E4F569900046E0FFE569C39F5027903A
:1042E600006AE475F001123227AFF0FE90003DE05F
:1042F600FD04F074042DF582E43400F583E0FD122C
:10430600374E056980CE7BFF7A06799D124D09905E
:05431600000074FEF040
:01431B00227F
:103CA00030216B900001E0FF900035F0C221121529
:103CB00012900035E0FFB42A079000007403F02250
:103CC0001254B4501A900035E0FF90003DE0FE041D
:103CD000F074042EF582E43400F583EFF080107B5D
:103CE000FF7A06797D124D0990000074FAF0229057
:103CF0000046E02409FFE433FE90003DE0D39FEE50
:0F3D00006480F87480984006900000E004F02280
:10333100900048E0FF70062027030233DC1215419C
:1033410012517590006AEEF0A3EFF012378F12124E
:10335100FC900046E0B40110900063E0FF121512EA
:10336100900063E0900024F0900046E0B4022090C9
:103371000062E0FF121512900063E0FF1215129037
:103381000062E0900024F0900063E0900025F0904E
:103391000046E064037030900061E0FF1215129066
:1033A1000062E0FF121512900063E0FF1215129007
:1033B1000061E0900024F0900062E0900025F09020
:1033C1000063E0900026F0302711C227900046E00C
:1033D100900034F090000074F0F02290004BE0FF78
:1033E10012154190003D740AF0900000E004F022B3
:10459D001213525002803B12132A8F6990004CE087
:1045AD00FFE569C39F402B90004DE0FFE569D39F68
:1045BD00502012517590006AEEF0A3EFF0AD691224
:1045CD00374E7BFF7A06799D124D0990000074FEDF
:0B45DD00F022124D0390000074FAF071
:0145E80022B0
:104417001213525002803F12132A8F6990004CE00A
:10442700FFE569C39F400B90004DE0FFE569D39F0F
:104437004004E569702012517590006AEEF0A3EF11
:10444700F0AD6912374E7BFF7A06799D124D0990C0
:0F445700000074FEF022124D0390000074FAF082
:014466002233
:1038E100900048E0FF700330275E121541125175B8
:1038F10090006AEEF0A3EFF012378F8F691237D87C
:10390100E4F56974612569F582E43400F583E0FF2B
:1039110074242569F582E43400F583EFF0746125A0
:1039210069F582E43400F583E0FF1215120569E5BB
:1039310069C3940440CD30270FC22790003474032B
:10394100F090000074F0F02290004BE0FF1215415E
:0C39510090003D740AF0900000E004F0CB
:01395D002247
:10481A007F0A122E328F69E5696012125175900073
:10482A006AEEF0A3EFF0E56914FD12374EE5697BF5
:10483A00FF600E7A06799D124D0990000074FEF011
:0E484A00227A06791D124D0990000074FAF0D2
:01485800223D
:1034B100900048E0FF700620270302354C121541A9
:1034C10012517590006AEEF0A3EFF012378F1212CD
:1034D100FC90006AE475F001123227AFF0FE12375A
:1034E1008F1212E0900062E0FF900024F0A3F0122E
:1034F1001512900063E0FF12151290006AE475F056
:1035010001123227AFF0FE12378F1212E0900061E4
:10351100E0FF900026F0900062E0900027F090001C
:1035210063E0900028F0121512900062E0FF12157E
:1035310012900063E0FF12151230270FC22790008E
:10354100347405F090000074F0F02290004BE0FF1D
:1035510012154190003D740AF0900000E004F02241
:1033F10090000EE0540F75F00AA4FFA3E0540F2FC4
:10340100F569900011E0540F75F00AA4FDACF0903D
:103411000010E0540F75F064A42DFFE5F03CFE9020
:103421000012E0540F7C002FFFEC3EFEE569C394CF
:10343100014019E569D394145012C3EF9401EE943D
:10344100004009D3EF94FAEE9400400A124D039024
:10345100000074FAF02212517590006AEEF0A3EFA9
:10346100F090006AE475F001123227AFF0FEAD6909
:1034710012374E900011E0540F75F00AA4FF90002E
:1034810010E0540F75F064A42FFF900012E0540F68
:103491002FF56990006AE0FEA3E0FFAD6912374E97
:0F34A1007BFF7A06799D124D0990000074FEF0B2
:0134B00022F9
:102293007F0D122E32EF701A900011E0B43010A3AC
:1022A300E0B4300BA3E0B43006A3E0643060030273
:1022B300238C900015E0FF64306004EFB4350E907A
:1022C3000016E0540FD39405400302238C900015AD
:1022D300E0FF64316004EFB4361190001AE0B420DB
:1022E30007900019E0B4200302238C900015E0FF4F
:1022F30064326004EFB43711900019E0B420079002
:102303000018E0B4200302238C900015E0FF64332F
:102313006004EFB43809900016E0B42002806A909C
:102323000015E0FF64346005EF64397066900016B1
:10233300E0540F75F00AA4FFA3E0540F2FF5699042
:102343000019E0540F75F00AA4FDACF0900018E0FA
:10235300540F75F064A42DFFE5F03CFE90001AE0E5
:10236300540F7C002FFFEC3EFEE569C39401401936
:10237300E569D394145012C3EF9401EE940040091D
:10238300D3EF94FAEE9400400A124D0390000074C8
:10239300FAF02212517590006AEEF0A3EFF090006C
:1023A3003D740AF0E4F569900046E0FFE569C39FD8
:1023B300502790006AE475F001123227AFF0FE90C7
:1023C300003DE0FD04F074042DF582E43400F58350
:1023D300E0FD12374E056980CE7BFF7A06799D12A8
:0823E3004D0990000074FEF0AA
:0123EB0022CF
:10395E00900048E0FF700330275B1215411251753D
:10396E0090006AEEF0A3EFF0E4F569900046E0FFF8
:10397E00E569C39F502C90006AE475F0011232275E
:10398E00AFF0FE12378F8F6A74242569F582E43406
:10399E0000F583E56AF07E0012378F121512056965
:1039AE0080C9302710C227E56904900034F09000DA
:1039BE000074F0F02290004BE0FF12154190003D94
:0B39CE00740AF0D224900000E004F026
:0139D90022CB
:103D7D00302165900001E0FF900035F0C221BF2A8F
:103D8D00079000007403F022900035E0FFB4230883
:103D9D00900000E004F0803DEF547FFF121512906B
:103DAD000035E0547FFF90003DE0FE04F074042EDA
:103DBD00F582E43400F583EFF0900046E02409FF2E
:103DCD00E433FE90003DE0D39FEE6480F87480985C
:093DDD004006900000E004F02211
:1044670030214B900001E0FF900035F0C221BF2AB8
:10447700079000007403F022900035E0FFB4230B8F
:10448700900000E004F0E004F080101254B4500FE4
:10449700900035E0900040F0900000E004F0227BAF
:0F44A700FF7A06797D124D0990000074FAF02219
:1036B10020210302374D900001E0FF900035F0C258
:1036C10021BF2A079000007403F022900035E0FF2B
:1036D100B4230A900000E004F0E004F0221254B494
:1036E100505B900040E0540F75F00AA4FF90003544
:1036F100E0540F2FF0E090089693FF900035F01200
:103701001512900035E0FF90003DE0FE04F07404D6
:103711002EF582E43400F583EFF0900046E02409B1
:10372100FFE433FE90003DE0D39FEE6480F87480A7
:1037310098900000E0400304F02214F0227BFF7A0D
:0D37410006797D124D0990000074FAF02207
:10506900301E09900077E0F561121206302003E442
:10507900F561301F0B301C0575610A8003756128C5
:07508900900000E004F0229A
:103DE600E5617063122F20900045E01232493E16BD
:103DF600643E1B6E3E1B783E1B823E1B8C3E20960D
:103E06003E25A03E2AAA3E2FB43E34BE00003E37D1
:103E160012535F801C124DC78017125597801212DD
:103E26005598800D125599800812559A800312559F
:103E36009B301E0D900076E0F55D900000E004F0EA
:083E4600229000007401F0223B
:0E54D200E55D700912120C9000007401F022CA
:10426E00301E0D900077E0F561121206E56170FCCC
:10427E00301F07756105E56170FCE4F569301F0CB0
:10428E0012553A1212AB12557A1212AB301E0C1294
:10429E0055451212AB12557A1212AB0569E569C378
:1042AE00940540D9301E0A900076E0F55DE55D700C
:0742BE00FC9000007401F008
:0142C50022D6
:0155930022F5
:0155940022F4
:0155950022F3
:103ACD00301F0A201C079000007401F022301E0DDB
:103ADD00900077E0F561121206E56170FC301F076A
:103AED00756105E56170FC301E1B90007EE0F537B9
:103AFD00125545E4F5691212AB0569E569C3940ADF
:103B0D0040F412557A301F1B90007FE0F5371255A7
:103B1D003AE4F5691212AB0569E569C3940A40F4FC
:103B2D0012557A301E0A900076E0F55DE55D70FC69
:083B3D001239DAE4900000F0F7
:013B4500225D
:0155960022F2
:10485900302F3B202138756264E53F547FFF900279
:104869005193900001F030240EE53F30E709EF90B5
:10487900026193900001F0D221C22F900001E0B4AF
:0F4889002307900002E004F022E4900002F022E6
:10489800302D3B202138756264E53D547FFF90023E
:1048A8005193900001F030240EE53D30E709EF9078
:1048B800026193900001F0D221C22D900001E0B472
:0F48C8002307900002E004F022E4900002F022A7
:101E5600202203021FC3302103021FC3900002E0A9
:101E6600F569E4F075626412558DD221BF30079092
:101E760000017430F022BF31079000017431F02266
:101E8600BF32079000017432F022BF330790000181
:101E96007433F022BF34079000017434F022BF354A
:101EA600079000017435F022BF36079000017436A2
:101EB600F022BF37079000017437F022BF38079031
:101EC60000017438F022BF39079000017439F022FE
:101ED600BF23109000017423F0AF690569900002DA
:101EE600EFF022BF2A07900001742AF022BF4107B3
:101EF6009000017441F022BF42079000017442F045
:101F060022BF43079000017443F022BF640790008C
:101F1600017444F022202403C22122BF61079000ED
:101F2600017461F022BF62079000017462F022BF63
:101F360063079000017463F022BF64079000017488
:101F460064F022BF65079000017465F022BF660742
:101F56009000017466F022BF67079000017467F075
:101F660022BF68079000017468F022BF69079000DD
:101F7600017469F022BF6A07900001746AF022BFFB
:101F86006B07900001746BF022BF6C079000017420
:101F96006CF022BF6D07900001746DF022BF6E07D2
:101FA600900001746EF022BF6F07900001746FF00D
:0D1FB60022BF70079000017470F022C2215C
:011FC30022FB
:0B550A007F209000047420F0A3DFFC61
:015515002273
:0F54B400EFC394304007EFD39439500122C32245
:103BBB0090000DE0FD6420602E90000CE0540F751A
:103BCB00F00AA4FBAAF090000BE0540F75F064A46C
:103BDB002BFFE5F03AFEED540F7C002FFFEC3E90EF
:103BEB000066F0A3EF803190000CE0FD64209000A4
:103BFB000B601AE0540F75F00AA4FFED540F7C0014
:103C0B002FFEEC35F0900066F0A3CE800BE0540F46
:103C1B00FF900066E4F0A3EFF0E024FFF090006665
:053C2B00E034FFF0226F
:103E4E0090000AE0FD6420602B900009E0540F758D
:103E5E00F00AA4FBAAF0900008E0540F75F064A4D9
:103E6E002BFFE5F03AFEED540F7C002FFFEC3E9059
:103E7E000068802E900009E0FD6420900008601A12
:103E8E00E0540F75F00AA4FFED540F7C002FFEECEA
:103E9E0035F0900068F0A3CEF022E0540FFF9000B2
:073EAE0068E4F0A3EFF0222D
:1051DC00900006E0540F75F00AA4FFA3E0540F2FC3
:1051EC00900036F0D394004006E09415500122C391
:0151FC002290
:10410100E4FFEF75F003A424ADF582E43406F583F2
:10411100E493FE900005E0FDEE6D703BEF75F0035A
:10412100A424AEF582E43406F583E493FE90000600
:10413100E0FDEEB50521EF75F003A424AFF582E4AF
:104141003406F583E493FE900007E0FDEEB5050724
:0C415100900037EFF0D3220FBF33A7C35C
:01415D00223F
:10404200E4FF75F003EFA42446F582E5F03407F5AA
:1040520083E493FE900005E0FDEE6D703D75F00384
:10406200EFA42447F582E5F03407F583E493FE904C
:104072000006E0FDEEB5052275F003EFA42448F535
:1040820082E5F03407F583E493FE900007E0FDEE4D
:0F409200B50507900038EFF0D3220FBF70A4C31D
:0140A10022FC
:102E320074042FF582E43400F583E0FD6431706997
:102E4200FE74052FF582E43400F583E0FCEE75F0A4
:102E520003A424ADF582E43406F583E4936C704256
:102E620074062FF582E43400F583E0FCEE75F0037E
:102E7200A424AEF582E43406F583E493B504237406
:102E8200072FF582E43400F583E0FCEE75F003A42D
:102E920024AFF582E43406F583E493B50404EE042A
:102EA200FF220EBE339B7F0022ED6432706DFE74F2
:102EB200052FF582E43400F583E0FD75F003EEA4FE
:102EC2002446F582E5F03407F583E4936D7045748A
:102ED200062FF582E43400F583E0FD75F003EEA4DD
:102EE2002447F582E5F03407F583E493B5052574AC
:102EF200072FF582E43400F583E0FD75F003EEA4BC
:102F02002448F582E5F03407F583E493B50505EE30
:0D2F12002434FF220EBE70977F00227F0046
:012F1F00228F
:1037D800EFC3943390006150397431F0EF75F00302
:1037E800A424ADF582E43406F583E493900062F0F6
:1037F800EF75F003A424AEF582E43406F583E49370
:10380800900063F0EF75F003A424AFF582E434066A
:10381800803A7432F075F003EFA424ADF582E5F038
:103828003406F583E493900062F075F003EFA42466
:10383800AEF582E5F03406F583E493900063F07505
:10384800F003EFA424AFF582E5F03406F583E493A2
:05385800900064F02265
:10537600900006E0540F75F00AA4FFA3E0540F2F27
:05538600900039F02247
:10538B00900006E0540F75F00AA4FFA3E0540F2F12
:05539B0090003AF02231
:1053A000900006E0540F75F00AA4FFA3E0540F2FFD
:0553B00090003BF0221B
:064D03007BFF7A0579ED4B
:064D09008B6A8A6B896CC5
:104D0F007F01121541E4F56DAB6AAA6BA96C856D35
:104D1F00827583001231A5FF121512056DE56DC363
:044D2F00941040E4B8
:014D3300225D
:064D34007BFF7A06793DC9
:064D3A008B6A8A6B896C94
:104D40007F11121541E4F56DAB6AAA6BA96C856DF4
:104D5000827583001231A5FF121512056DE56DC332
:044D6000941040E487
:014D6400222C
:10517500900050E0FF90004FE08FF0A4FF90004EAC
:10518500E07C002FFFEC35F0FE900047E02FFFECB0
:035195003EFE22B9
:1053B500900049E075F010A42423F9740A35F0FA39
:0553C5007BFF024D3AE0
:03558D007F032277
:104FC100124AEEE4F569AF697E00E569900CF3934E
:104FD100FD12374EAF697E00E569900CF393FD1227
:0B4FE10046C70569E569C3942540DB65
:014FEC0022A2
:10326F00E4F569AF697E0012378F746C2569F582BA
:10327F00E43400F583EFF00569E569C3942540E375
:10328F0090006CE0F520E5205440900091F0900004
:10329F007CE0F53490007BE0FF7008F58453BCF8B8
:1032AF0043BC06EFB40106E4F58453BCF8EFB40257
:1032BF0009E4F58453BCF843BC01EFB40309E4F50A
:1032CF008453BCF843BC02EFB40409E4F58453BC47
:1032DF00F843BC03EFB40509E4F58453BCF843BCD1
:1032EF000490007AE0FF7009758402E5BC54FCF588
:1032FF0042EFB4010C758402E5BC54FCF542434225
:10330F0001EFB4020C758402E5BC54FCF542434254
:10331F0002EFB4030C758402E5BC54FCF542434242
:01332F00039A
:01333000227A
:10535F00301E08900024E0FF125522301F089000E5
:07536F0024E0FF1255162295
:104DC700E4F569900034E0FFE569C39F502174243E
:104DD7002569F582E43400F583E0F56A301E04FFA7
:0F4DE700125522301F05AF6A125516056980D488
:014DF600229A
:0155970022F1
:0155980022F0
:0155990022EF
:01559A0022EE
:01559B0022ED
:0C5516001255501212AB1255810212AB5C
:0C55220012555B1212AB1255810212AB45
:102F2000E4F569F56AF56B900067E02401FF900015
:102F300066E03400FEC3EF940AEE94005005A3E06F
:102F400004F56BD3EF9463EE9400404C900067E07F
:102F50002401FB900066E03400FA7C007D64AF033E
:102F6000FE1231D28F69EF75F064A4FFC3EB9FFFAF
:102F7000EA95F0FE7C007D0A1231D28F6AA3E0044C
:102F8000FFE56975F064A4FEC3EF9EFFE56A75F086
:102F90000AA4FEC3EF9EF56B900067E02401FF904A
:102FA0000066E03400FED3EF9409EE940040197CF3
:102FB000007D0A1231D28F6AA3E004FFE56A75F042
:102FC0000AA4FEC3EF9EF56B74302569F569743071
:102FD000256AF56A7430256BF56B301E14AF6912E3
:102FE0005522AF6A125522AF6B1255227F2A125515
:102FF00022301F14AF69125516AF6A125516AF6B07
:083000001255167F2A12551625
:0130080022A5
:1030D900E4F569F56AAF6AAE69124EDD746C256A6A
:1030E900F582E43400F583EFF0056AE56A700205BC
:1030F90069C39425E569940040DB90006CE0F520F4
:10310900E5205440900091F090007CE0F534900067
:103119007BE0FF7008F58453BCF843BC06EFB401AB
:1031290006E4F58453BCF8EFB40209E4F58453BC12
:10313900F843BC01EFB40309E4F58453BCF843BC7C
:1031490002EFB40409E4F58453BCF843BC03EFB4BB
:103159000509E4F58453BCF843BC0490007AE0FF08
:103169007009758402E5BC54FCF542EFB4010C7595
:103179008402E5BC54FCF542434201EFB4020C75EC
:103189008402E5BC54FCF542434202EFB4030C75DA
:0B3199008402E5BC54FCF542434203F5
:0131A4002208
:104FED00E4F569F56A746C256AF582E43400F5839D
:104FFD00E0FDAF6AAE6912374E056AE56A700205CB
:0A500D0069C39425E569940040DBB7
:015017002276
:10501800124AEEE4F569F56AAF6AAE6912378FADE8
:1050280007AF6AAE691246C7056AE56A7002056984
:09503800C39425E569940040DFF2
:01504100224C
:10360A00535155452020434F53202053454E53458F
:10361A00004F4E2020202020202020202020202063
:10362A0020004F4646202020202020202020202035
:10363A002020002A2A3132333435362A2A2A2A31DE
:10364A0032333435302A2A44313233343536373836
:10365A0039302A2341424356455253494F4E204D51
:10366A00495820312E30312020434F5320414354B2
:10367A004956452020202020535155454C43482087
:10368A0041435449564520202053454E5345204135
:10369A004354495645202053494D504C45582052D1
:0736AA004550454154455213
:10356100302825C228E53F540F903651939000A58D
:10357100F0123F19754E32900097E004F0300114BB
:10358100124C021249C9800CE54E7008900092F06D
:103591009000A2F030293DC229E53D540F903651EB
:1035A100939000A4F0123EB5754F32900097E0045D
:1035B100F0301C03200006201C0630020312498E45
:1035C100301C03200003201C03124BCD201C1112C0
:1035D1004C9F800CE54F7008900093F09000A1F093
:1035E100302319300322123EB57550321255909096
:1035F1000096EFF0C223124A04024C37E5507008DE
:09360100900094F09000A3F02267
:104BCD00900093E0FF04F0EF90363D93FF9000A42A
:104BDD00E0FEEF6E6011EEB42A089000937401F0C0
:104BED008005E4900093F0900093E0B40A06E4F0A1
:054BFD00D21FD22A22A4
:104C0200900092E0FF04F0EF90363D93FF9000A5F4
:104C1200E0FEEF6E6011EEB42A089000927401F08B
:104C22008005E4900092F0900092E0B40A06E4F06D
:054C3200D21ED22A226F
:104C3700900094E0FF04F0EF90363D93FF900096CC
:104C4700E0FEEF6E6011EEB42A089000947401F054
:104C57008005E4900094F0900094E0B40A06E4F034
:054C6700D220D22A2238
:10498E009000A1E0FF04F074982FF582E43400F556
:10499E0083E0FF9000A4E0FEEF6E6011EEB42308FA
:1049AE009000A17401F08005E49000A1F09000A1A8
:0B49BE00E0B40906E4F0D21FD21D2275
:1049C9009000A2E0FF04F074982FF582E43400F51A
:1049D90083E0FF9000A5E0FEEF6E6011EEB42308BE
:1049E9009000A27401F08005E49000A2F09000A26A
:0B49F900E0B40906E4F0D21ED21D223B
:104A04009000A3E0FF04F074982FF582E43400F5DD
:104A140083E0FF900096E0FEEF6E6011EEB4230891
:104A24009000A37401F08005E49000A3F09000A32B
:0B4A3400E0B40906E4F0D220D21D22FD
:104C9F00900095E0FF04F0EF90364793FF9000A44B
:104CAF00E0FEEF6E6011EEB42A089000957401F0EB
:104CBF008005E4900095F0900095E0B40A04E4F0CC
:034CCF00D22B22C3
:104F67009000987423F0A3F0E4FF746D2FF582E4AA
:104F77003400F583E0FE749A2FF582E43400F5835C
:0C4F8700EEF00FBF06E49000A07423F0D1
:014F930022FB
:1039DA0012146F12155B12156A7F011215417BFFD3
:1039EA007A3679A1124D097BFF7A367961124D3AFE
:1039FA00755F14E4900097F07F10900051E4F0A3F3
:103A0A00DFFC7F10E55F70FC12521E500C7BFF7AC0
:103A1A00367971124D09755F14E55F70FC12123424
:103A2A00400C7BFF7A367981124D09755F14E55F88
:103A3A0070FC12523E500C7BFF7A367991124D0976
:0A3A4A00755F14E55F70FC02155B68
:103EB500900097E0FED3940F50129000A4E0FF7499
:103EC500512EF582E43400F583EF80437F0112150E
:103ED50041E4F56974522569F582E43400F583E01F
:103EE500FF74512569F582E43400F583EFF07451D0
:103EF5002569F582E43400F583E0FF1215120569A2
:103F0500E569C3940F40CD9000A4E0FF900060F0F8
:033F150012151270
:013F18002286
:103F1900900097E0FED3940F50129000A5E0FF7433
:103F2900512EF582E43400F583EF80437F011215A9
:103F390041E4F56974522569F582E43400F583E0BA
:103F4900FF74512569F582E43400F583EFF074516B
:103F59002569F582E43400F583E0FF12151205693D
:103F6900E569C3940F40CD9000A5E0FF900060F093
:033F79001215120C
:013F7C002222
:035590007F012276
:103FE1007BFF7A36790A124D091212347BFF4006A3
:103FF1007A36791B80047A36792C124D3A7F171262
:104001001541AF321212FC900061E0FF12151290BF
:104011000062E0FF121512900063E0FF1215127F9B
:104021001C121541AF311212FC900061E0FF121514
:1040310012900062E0FF121512900063E0FF02157A
:01404100126C
:1030090020202020202020202020202020202020B7
:10301900205741495420464F5220544F4E452020B5
:10302900205741495420464F5220564F4943452085
:103039002020584D542054574F20544F4E4520209E
:1030490020202020584D5420564F49434520202008
:10305900205245434F5244494E4720564F49434514
:1030690020504147494E47204F4E4C59202020209F
:10307900202020535455434B204D494B45202020B7
:103089002056455253494F4E20312E3320202020BF
:1030990042555359205854524D4348414E4E454C80
:1030A900202020434F532041435449564520202096
:1030B9002020434F5320494E41435449564520202F
:1030C90020504C41594241434B2044454C415920E1
:102D0B0012155B9000A7E01232492DAC002DAF01DC
:102D1B002DB2022DB5032DB8042DBB052DBE062DEE
:102D2B00C1072DC4082DC7092DCA0A2DCD0B2DD0D7
:102D3B000C2DD3142DD6152DD8162DDA172DDC18F6
:102D4B002DDE192DE01A2DE21B2DE41C2DE61D2D79
:102D5B00E81E2DEA1F2DEC202DEE212DF0222DF259
:102D6B00282DF5292DF82A2DFB2B2DFE2C2E01328B
:102D7B002E04332E07342E0A352E0D362E10372EF9
:102D8B0013382E16392E193A2E1C3B2E1F3C2E2291
:102D9B003D2E253E2E283F2E2B402DF04100002EA0
:102DAB003102515102544F024F94024D650254E0CF
:102DBB00025473024E250253CA024E530253DD02D4
:102DCB0053F0025105025090024A7A802F803080D6
:102DDB003180328033803480358036803780388044
:102DEB0039803A803B803C024EAF0248D70254C335
:102DFB0002532902527D0251FD0252D6024AB402FD
:102E0B00530E024A3F024D960254EE025484024E78
:102E1B00810254030251980254160254290251BAEA
:072E2B0002512B1250B722E7
:10515100900085E07BFF700E7A307929124D3A90EC
:1051610000A77401F0227A307919124D3A9000A704
:045171007414F022A0
:10544F00125566500C900080E0F55E9000A7E004C6
:02545F00F02239
:104F9400E55E701DF54BF54C900073E0F55C9000F8
:104FA40081E0F55F900074E0F5609000A7E004F004
:0D4FB4002212557040069000A7E014F02274
:104D6500125570500A900081E0F55FD2088002C2AA
:104D750008121B3D501A7BFF7A307959124D3AE5DE
:104D85005C6004E55F7009E4F54B9000A7E004F072
:014D950022FB
:0E54E000C208121B8650069000A7E004F022BE
:10547300E5606006E49000A7F0229000A7E004F046
:015483002206
:104E250090008FE0700D900090E0F5669000A7E08F
:104E350004F02212521E400C900090E0F56690009E
:0E4E4500A7E004F07BFF7A307999124D3A22F3
:1053CA00E56670069000A7E004F07BFF7A3079C9A1
:0353DA00024D3A47
:104E530090008FE0700D900090E0F5669000A7E061
:104E630004F02212521E400C900090E0F566900070
:0E4E7300A7E004F07BFF7A307999124D3A22C5
:1053DD00900075E0F55B1212121212069000A7E014
:0353ED0004F022A7
:1053F000E55B700EF54B900073E0F55C9000A7E064
:0354000004F02293
:10510500C20AD2127BFF7A307949124D3A121ACF70
:105115004004E55C700FE4F54B900076E0F55D909A
:0651250000A7E004F022E7
:10509000C20AC212121B86501DE55D701912120C55
:1050A0001212187BFF7A307979124D3A12557040FE
:0750B00005E49000A7F022C7
:104A7A0012523E501A900083E0FF700D900080E0C1
:104A8A00F55E9000A77432F0228F59C218801490F4
:104A9A000085E0B4021312521E500E900083E0F516
:0A4AAA0059D2189000A7E004F02292
:104AB400E5597035900084E0701A900043F090003E
:104AC40083E0F5597BFF7A307969124D3A9000A75B
:104AD4007428F022900084E0F55A7BFF7A3079291B
:0A4AE400124D3A9000A7E004F02202
:10530E00125566500D900080E0F55E9000A7E00407
:0B531E00F022E55A70049000A7F02276
:104A3F00E55E7022F54BF54C900073E0F55C90004D
:104A4F0081E0F55F900074E0F560E4900043F09032
:104A5F0000A7E004F02212557040079000A7E01461
:0B4A6F00F022E55A70049000A7F0222E
:104D9600125570500A900081E0F55FD2088002C279
:104DA60008121B3D501A7BFF7A307959124D3AE5AD
:104DB6005C6004E55F7009E4F54B9000A7E004F041
:014DC60022CA
:0E54EE00C208121B8650069000A7E004F022B0
:10548400E5606006E49000A7F0229000A7E004F035
:0154940022F5
:104E810090008FE0700D900090E0F5669000A7E033
:104E910004F02212521E400C900090E0F566900042
:0E4EA100A7E004F07BFF7A307999124D3A2297
:10540300E56670069000A7E004F07BFF7A3079C967
:03541300024D3A0D
:1051980090008FE070079000A7E004F02212521EE2
:1051A80040069000A7E004F07BFF7A307999124D11
:0251B8003A2299
:10541600900075E0F55B1212121212069000A7E0DA
:0354260004F0226D
:10542900E55B700EF54B900073E0F55C9000A7E02A
:0354390004F0225A
:1051BA00E55B701D7BFF7A307939124D3A120F95F3
:1051CA00500F900073E0F55CE4F54B9000A7E00403
:0251DA00F022C1
:10512B00C20AD2127BFF7A307949124D3A121ACF4A
:10513B004004E55C700FE4F54B900076E0F55D9074
:06514B0000A7E004F022C1
:1050B700C20AC212121B86501DE55D701912120C2E
:1050C7001212187BFF7A307979124D3A12557040D7
:0750D70005E49000A7F022A0
:104EAF0075700190008FE0600812521E5003E4F5F8
:104EBF0070E5597010E570600C900090E0F5669009
:0E4ECF0000A7E004F07BFF7A307999024D3A9B
:1048D70075700190008FE0600812521E5003E4F5D6
:1048E70070E5667016E5706012900075E0F55B1272
:1048F70012121212069000A7E004F0E5667BFF6033
:0F490700067A3079C980047A307999124D3A22B4
:0F54C300E55B700A900043F09000A7E004F02230
:105329007BFF7A307939124D3A120F95500C900063
:0B53390076E0F55D9000A7E004F02294
:10527D00E55D701912120C1212187BFF7A307979D4
:0E528D00124D3A1255704005E49000A7F02231
:1051FD00E55E701C12521E400E9000A7E004F07B7D
:10520D00FF7A3079B980067BFF7A3079A9124D3A51
:01521D00226E
:1052D60012521E500D9000A7E004F0900083E0F5F6
:0C52E60059227BFF7A307929124D3A22C0
:101AB400754B00121AFD50FB22754B00121B865009
:101AC400FB22754B00121B3D50FB22758400E54B35
:101AD40075F003A4901ADC73021BA2021BB1021B53
:101AE400CF021BB8021BDB021BE2021BEA021BB182
:101AF400021BF8021BB8021C3D758400E54B75F00F
:101B040003A4901B0A73021BA2021BB1021BCF0287
:101B14001BB8021BDB021BE2021BEA021BB1021B05
:101B2400F8021BB8021C08021C11021BA2021BB102
:101B3400021C1F021BB8021C2B758400E54B75F0B8
:101B440003A4901B4A73021BA2021BB1021BCF0207
:101B54001BB8021BDB021BE2021BA2021BB1021B0D
:101B6400CF021BB8021BDB021BE2021BDB021BE2DF
:101B7400021BEA021BB1021C2D021BB8021C080244
:101B84001C2B758400E54B75F003A4901B93730222
:101B94001BA2021BB1021C1F021BB8021C2BC2FA9F
:101BA400121C47121C47759B00054BC32230F902D7
:101BB400054BC32230F912E59A20E7FB121C47D2E9
:101BC400FA121C47121C47054BC322C2FA121C47C7
:101BD400759B04054BC322752E1E054BC322E52EAF
:101BE4007002054BC322C2FA121C47121C68F59BF3
:101BF400054BC322C2FA121C47121C774407F59BFB
:101C0400054BC322121C59F52F054BC32275840FB3
:071C140030DE04E52F700231
:101C1B00054BC322C2FA121C47759B08054BC32206
:101C2B00D322C2FA121C47121C774405F59B054BB5
:101C3B00C32275840F30DE02C322D32200000000C2
:101C4B000000000000000000000000000022901CBB
:101C5B0060E54C93225A5A5A5A5AFAFAFA901C6F68
:101C6B00E54C932200B45AE12D877ADB901C7EE57C
:0B1C7B004C932200000000000080805D
:10385D0075840F1200A41230D9124FED124F67125A
:10386D0039DA12120C20A605123FE1800B30A705A4
:10387D00122D0B800312415E123561123F7D302AED
:10388D0036C22A7F0C121588E4FF12158E124FC115
:10389D0012326F124F67C21EC21FC220E4F56812AA
:1038AD0012AB0568E568C3941E40F41239DAE49052
:1038BD0000A7F09000A8F0301DAB124C6C12326FC7
:1038CD00124F67C21EC21FC220E49000A7F09000E5
:0438DD00A8F080913E
:103F7D00900041E0701412124F400F12121E756521
:103F8D006412553A900041E004F0900041E0B40114
:103F9D0010E565703E12557A75643C900041E00461
:103FAD00F0900041E06402701E1212615005121271
:103FBD005B4007E5647010201D0D121226756564B7
:103FCD00900041E004F022900041E0B40305E56566
:043FDD007001F0225D
:101C860009920A9E0BC70D100E7D101211D213C5B4
:101C960015ED185208D0094E09D40A600AF40B91C2
:101CA6000C360CE50D9D0E600F2D100610EB11DDA8
:101CB60012DC13EA15071633177118C01D2107B178
:101CC60007E808200859196E1A211ADA1B971C5AB8
:101CD6000894090E09900A190AA90B410BE30C8C0A
:101CE6000D3F0DFD0EC50F9810771162125B136242
:101CF6001477159B16D018161DEF1EC21F9B207950
:101D0600215F224A233B24342533263912330FCD53
:101D160014331566169A17CD19000E9A136611001C
:101D260011661033150016331766189A19CD0DCDA6
:101D36000F00129A11CD1300149A15CD17001833FF
:101D460019660E330F66109A078607DC0835089267
:101D560008F3095909C30A320AA50B1E0B9C0C1F6E
:101D66000CA90D390DCF0E6B0F0F0FBA106C112584
:101D760011EB12B113851466154E163D173A184429
:101D860019551A741BA01CDA1E221F7720DA22525C
:101D960023D7256A271128CD2A9D2C822E7B3088B1
:101DA60032B134EF374739B53C443EF641BB44AA1D
:101DB60047AE4ADA4E2F51A75541590A5CFC181610
:101DC6001DEF1EC21F9B2079215F224A233B24342C
:101DD6002533263912330FCD14331566169A17CDCF
:101DE60019000E9A1366110011661033150016338A
:101DF6001766189A19CD0DCD0F00129A11CD130042
:101E0600149A15CD1700183319660E330F66109AFB
:101E1600191823A01296203D129623A01296276326
:101E26001488203D148823A01488276316B8203D03
:101E360016B823A016B827631918203D191827636A
:101E460012962B8C14882B8C16B82B8C19182B8C6D
:100F950090007DE0F537900043E0FF600302102AE2
:100FA500301832900091E090008B7010E0540F756E
:100FB500F014A42486F582E4341C800EE0540F75E9
:100FC500F014A4244EF582E4341DF583C083C08259
:100FD50090008C8030900091E09000877010E05474
:100FE5000F75F014A42486F582E4341C800EE054B9
:100FF5000F75F014A4244EF582E4341DF583C083E7
:10100500C082900088E0540FD082D08375F0021220
:10101500323DE493F508740193F509D231D2137585
:10102500630A0211ECEF640160030211F4E56360E9
:1010350002C32275631E20180302111B900091E064
:10104500706A90008DE0540F75F014A42486F58223
:10105500E4341CF583C083C08290008EE0540FD029
:1010650082D08375F00212323DE493F50874019342
:10107500F50990008BE0540F75F014A42486F582D1
:10108500E4341CF583C083C08290008CE0540FD0FB
:1010950082D08375F00212323D74019365097004A4
:1010A500E493650860030211EC0211E990008DE0FC
:1010B500540F75F014A4244EF582E4341DF583C055
:1010C50083C08290008EE0540FD082D08375F002E9
:1010D50012323DE493F508740193F50990008BE015
:1010E500540F75F014A4244EF582E4341DF583C025
:1010F50083C08290008CE0540FD082D08375F002BB
:1011050012323D74019365097004E4936508600328
:101115000211EC0211E9900091E07066900089E0FF
:10112500540F75F014A42486F582E4341CF583C0AD
:1011350083C08290008AE0540FD082D08375F0027C
:1011450012323DE493F508740193F509900087E0A8
:10115500540F75F014A42486F582E4341CF583C07D
:1011650083C082900088E0540FD082D08375F0024E
:1011750012323D74019365097004E4936508706744
:101185008062900089E0540F75F014A4244EF58216
:10119500E4341DF583C083C08290008AE0540FD0EB
:1011A50082D08375F00212323DE493F50874019301
:1011B500F509900087E0540F75F014A4244EF582CC
:1011C500E4341DF583C083C082900088E0540FD0BD
:1011D50082D08375F00212323D740193B50908E49B
:1011E50093B50803756346900043E004F0C322906D
:1011F5000043E0B4020AE5636002C32212557AD3C4
:0112050022C6
:0B553A0075081575095ED231D20B22F6
:0B55450075081575095ED231D21322E3
:07557A00C231C20BC2132273
:0B55500090007812212FD232D20C22E2
:0B555B0090007912212FD232D21422CE
:0C212F00E0F536E4F512F513F514F51593
:10213B00EF12324922362322252A21733021853191
:10214B0021973221A93321BB3421CD3521DF362113
:10215B00F13722033822143922474122584222698F
:10216B0043227A4400002292901E16E493F50D74DC
:10217B000193F50E901E18022289901E1AE493F516
:10218B000D740193F50E901E1C022289901E1EE405
:10219B0093F50D740193F50E901E20022289901E6B
:1021AB0022E493F50D740193F50E901E24022289FF
:1021BB00901E26E493F50D740193F50E901E2802E4
:1021CB002289901E2AE493F50D740193F50E901E4F
:1021DB002C022289901E2EE493F50D740193F50EBB
:1021EB00901E30022289901E32E493F50D740193F8
:1021FB00F50E901E34022289901E36E493F50D7471
:10220B000193F50E901E388075901E3AE493F50DF0
:10221B00740193F50E901E3C8064901E3EE493F582
:10222B000D740193F50E901E408053901E42E49363
:10223B00F50D740193F50E901E448042901E46E4FA
:10224B0093F50D740193F50E901E488031901E4A44
:10225B00E493F50D740193F50E901E4C8020901EA7
:10226B004EE493F50D740193F50E901E50800F9074
:10227B001E52E493F50D740193F50E901E54E493E6
:08228B00F50F740193F5102218
:07558100C232C214C20C2269
:1046C700AC84A2AF9238ABB1C2AF75840F53A1FED1
:1046D70075B121E4F58443B701F584438F0178A1CF
:1046E700768008F6EF26F618EE36F6E6FE08E6F5CB
:1046F700828E83EDF0E4F584538FFEF58453B7FE85
:084707008BB18C84A23892AF43
:01470F002287
:104EDD00AD84A2AF9238ACB1C2AF75B121756E8001
:104EED00756F00EF256FF56FEE356EF56E856F8280
:0D4EFD00F583E493FF8CB18D84A23892AF51
:014F0A002284
:104AEE00AF84A2AF9238AEB1C2AF78A1768008760D
:104AFE000075B121E4F58443B701F584758F031871
:104B0E00E6FC08E6F5828C83E4F0F58FF58453B766
:094B1E00FE8EB18F84A23892AF23
:014B2700226B
:103C30002020202020202020202020202020202084
:103C4000202052454345495645204D4F44452020AC
:103C5000202020205245434F5244494E47202020E7
:103C600042555359205854524D4348414E4E454CAD
:103C7000205741495420464F522053454E5345202A
:103C800020205452414E534D495454494E47202010
:103C9000202020535455434B204D494B4520202094
:10415E0012155B9000A8E0B40C00504F904171F81E
:10416E0028287302419502419802419B02419E020A
:10417E0041A10241A40241A70241AA0241AD02415E
:10418E00B00241B30241B6025495025461024B97FC
:10419E000249160254FC02543C024F0B02529B027F
:0C41AE0053440252F20252B91250DE22B9
:105495007BFF7A3C7940124D3A9000A87401F022C6
:10546100125566500C900080E0F55E9000A8E004B3
:02547100F02227
:104B9700E55E7026F54BF54C900073E0F55C9000F0
:104BA70081E0F55F900074E0F5607BFF7A3C795017
:104BB700124D3A9000A8E004F0221255704006907A
:064BC70000A8E014F0223A
:104916001255705010900081E0F55F900084E0F52C
:104926005AD2088002C20812523E50069000A9745C
:1049360001F0121B3D5015E55C6008E55A700DE567
:0D4946005F7009E4F54B9000A8E004F0223A
:0E54FC00C208121B8650069000A8E004F022A1
:10543C00E5606008E49000A8F0A3F0229000A8E0DA
:03544C0004F02247
:104F0B0090008FE0700D900090E0F5669000A8E0A7
:104F1B0004F02212521E400C900090E0F5669000B7
:0E4F2B00A8E004F07BFF7A3C7960124D3A2238
:10529B007BFF7A3C7970124D3A9000A9E06009E4EB
:0E52AB00F09000A8E004F022E49000A8F022A9
:10534400E5667016F54BF54C900075E0F55B1212AE
:0B535400121212069000A8E004F022E4
:1052F200E55B7017F54B900073E0F55C7BFF7A3C41
:0C5302007980124D3A9000A8E004F022DF
:1052B900C20AD212121ACF4004E55C700FE4F54B12
:0D52C900900076E0F55D9000A8E004F02272
:1050DE00C20AC212121B86501DE55D701912120C07
:1050EE001212187BFF7A3C7990124D3A125570408D
:0750FE0005E49000A8F02278
:10521E0030050F900082E0FFE532D39F4002D3228B
:10522E00C322900082E0FFE532C39F500122C322C9
:05558800121234B322F1
:10523E0030070F900086E0FFE531D39F4002D32266
:10524E00C322900086E0FFE531C39F500122C322A6
:104F3900300511900082E024F9FFE532D39F400249
:104F4900D322C322900082E02407FFE433FEC3E5A5
:0E4F5900329FEE6480F8748098500122C322CB
:0A55660030040302558812521E2281
:0A557000300403025588124F39225F
:0300000002552E78
:0C552E00787FE4F6D8FD7581A202385D9C
:1031A500BB010CE58229F582E5833AF583E02250DF
:1031B50006E92582F8E622BBFE06E92582F8E22229
:0D31C500E58229F582E5833AF583E4932243
:1031D200BC000BBE0029EF8DF084FFADF022E4CCE1
:1031E200F875F008EF2FFFEE33FEEC33FCEE9DECAA
:1031F200984005FCEE9DFE0FD5F0E9E4CEFD22EDF0
:10320200F8F5F0EE8420D21CFEADF075F008EF2F39
:10321200FFED33FD4007985006D5F0F222C398FD2A
:053222000FD5F0EA22C7
:10322700A3F8E0C5F025F0F0E5821582700215835A
:06323700E0C838F0E822B7
:0C323D00A42582F582E5F03583F583229C
:10324900D083D082F8E4937012740193700DA3A314
:1032590093F8740193F5828883E473740293686028
:06326900EFA3A3A380DF28
:00000001FF
